:100000000BC01895189518951895189522C1189534
:1000100018951895189518958FED8DBFC0ECE8EBE5
:100020004E2EDD275D2EEEE7F0E0A0E6B0E088275B
:100030008D933197E9F784B7082E877F84BF8FE1CE
:1000400081BD87E081BD662487EF8ABB8FE087BBD7
:1000500088E08BBB8FE088BB86E886B980E887B9EB
:1000600082E083BF789489B7826089BF82E083BFD2
:10007000E4E6F4E0FCD181E090E0A9E68D939C9366
:10008000A9E60D911C910A3050E0150710F009F017
:100090000CC0F0D1A9E6AD90AAE6AA0D1FD30C9230
:1000A000E6D1A9E6EAD108F4EBCF80E080936000C6
:1000B00080E080936100A9E71ED3809183008F7B4D
:1000C00080938300A3E88C9187FB0EF0C1C08091E0
:1000D00083008F778093830000916200003009F0E5
:1000E00035C0C09AADE70D911C9141E050E0040F7E
:1000F000151FA9E60D931C93A9E6AD90AAE6AA0DDB
:100100008C918BBBC19AC398A3E88C9186FB0EF0AF
:100110001DC0A9E70D911C9144E650E0DAD1A1E899
:100120004D935C93A1E80D911C9144E650E0EBD116
:10013000A9E60D931C93A9E70D911C91A9E64D9199
:100140005C91041B150BA5E70D931C9300916200B5
:10015000013009F03CC0A3E88C9185FB0EF402C08D
:10016000C09801C0C09AAFE70D911C9141E050E0EA
:10017000040F151FA9E60D931C93A9E6AD90AAE6FE
:10018000AA0D8C918BBBC39AC298A3E88C9186FB75
:100190000EF01DC0A5E70D911C914AE050E099D1E9
:1001A000AFE74D935C93AFE70D911C914AE050E0AF
:1001B000AAD1A9E60D931C93A5E70D911C91A9E680
:1001C0004D915C91041B150BA7E70D931C930091B7
:1001D0006200023009F03CC0A3E88C9185FB0EF070
:1001E00002C0C09801C0C09AA1E80D911C9141E0E5
:1001F00050E0040F151FA9E60D931C93A9E6AD90DE
:10020000AAE6AA0D8C918BBBC29AC198A3E88C91E7
:1002100086FB0EF01DC0A7E70D911C9141E050E058
:1002200058D1ADE74D935C93ADE70D911C9141E042
:1002300050E069D1A9E60D931C93A7E70D911C919D
:10024000A9E64D915C91041B150BABE70D931C9334
:1002500039CF0F921F922F923F924F925F927F92CF
:10026000AF92BF920F931F932F933F934F935F9340
:100270006F937F938F939F93AF93BF93CF93DF93AE
:10028000EF93FF938FB78F93A0E68C918F5F8C9342
:1002900000916000063010F009F001C0C7C080E096
:1002A0008093600080918300806880938300A2E641
:1002B0008C918F5F8C9300916200023010F009F0F6
:1002C00001C008C080E080936200809183008F7B32
:1002D00080938300A1E68C918F5F8C9300916100E5
:1002E0000E3110F009F001C0A1C080E080936100E0
:1002F00080918300806480938300CB9B09C08091B0
:1003000083008F7D8093830087E08093840008C002
:100310008091830080628093830089E180938400D0
:10032000379AEF93FF93E4ECF0E000D1FF91EF9167
:1003300007B1007EA4E88C9190E0890F082707B9E7
:10034000FED0A3E68D939C933798A3E696D0E3E680
:10035000F0E0D190E080FF2400274DD1A5E67CD1CC
:10036000E2E1F7E0BFD1E5E6F0E026D187D1EDE0AC
:10037000A5E6C9D1A3E88C9185FB0EF40BC0E6E19C
:10038000F7E0B0D1E5E6F0E017D178D1EDE0A5E6F1
:10039000BAD146C0A3E60D911C91093050E0150773
:1003A00008F00AC0EAE1F7E09DD1E5E6F0E004D10B
:1003B00065D1EDE0A5E6A7D1A3E60D911C9109302A
:1003C00050E0150781E008F480E08F93A3E60D91DB
:1003D0001C91053450E0150781E008F080E09F9102
:1003E0008923882309F40AC0EEE1F7E07BD1E5E632
:1003F000F0E0E2D043D1EDE0A5E685D1A3E60D9192
:100400001C91053450E0150708F40AC0E2E2F7E059
:1004100069D1E5E6F0E0D0D031D1EDE0A5E673D1C9
:10042000E5E6F0E095D0A9E7DD92EC928F918FBFE1
:10043000FF91EF91DF91CF91BF91AF919F918F91FC
:100440007F916F915F914F913F912F911F910F91EC
:10045000BF90AF907F905F904F903F902F901F90F4
:100460000F90189509CF2A4ACC581CCB08C88E2E5D
:100470009F2E0895E82DF92D0895ED91FC91EF5FE1
:10048000FF4FFC93EE93089508D03DD000FC10D0B0
:10049000089503D01ED001F8F9CF0024E89457FF47
:1004A00002C009D0689400F80BD010F80124089518
:1004B00002D009D00895509540954F5F5F4F089541
:1004C000E89417FF0895009510950F5F1F4F6894EB
:1004D0000895352F242FE894452B11F4689408953E
:1004E000512F402F0027112780E1440F551F001F77
:1004F000111F021B130B416018F4020F131F4E7FD4
:100500008A9599F70895752F642F55274427FF93EF
:10051000F1E1889405C010F4460F571F5695479592
:1005200017950795FA95B9F7FF9108953197F1F767
:100530000895689462F80895E89462F80895369AE8
:100540003699FECF369A3699FECF84B195B108958B
:1005500033D0992711278F2D880F80E8F82A802F14
:10056000881F08F41FEF41F08F57082F07FD04C0C4
:10057000003240F08FEF01C08827982FD82EE82E48
:10058000F82E09C08FE1801B082FF694E794D794CA
:1005900097950A95D1F7112351F09095D094E09456
:1005A000F09481E0980F8827D81EE81EF81E0F2DC2
:1005B000FE2CED2CD92E0895D190E190F19001916F
:1005C0000895102F90E8FF0C001F0927990FF7944A
:1005D0001078652F90E8440F551F5927990F4795BC
:1005E000607800380895FF0C90E89027110F9795D8
:1005F000F794092F0895102FBD2CDE2CEF2CF02E30
:1006000011234AF4B094D094E094F0949FEFB91A77
:10061000D90AE90AF90A0EE1FF2039F4FE2CED2C83
:10062000DB2CBB240850C2F723C032F00A95BB0C68
:10063000DD1CEE1CFF1CF9CF01D0D5CFB7FE08950D
:1006400090E8B91611F4D0FE08959FEFD91AE90A7F
:10065000F90A09F403950895DD92ED92FD920C9349
:1006600008959FE7092FF92A9FEFD92EE92E0895C3
:10067000DD24EE24FF24002711270895A2DFC1F313
:100680005038B1F31627005850580894051F12F43B
:1006900018F4E7CF08F0ECCF0AD0FF202AF0BB0C0B
:1006A000DD1CEE1CFF1C9FCF0F5FDBF29CCF9F92E7
:1006B0009924AA24BB24992788E1990CAA1CBB1C65
:1006C000DD1CEE1CFF1C30F4920EA31EB41ED91EBE
:1006D000E91EF91E8A9589F79F900895C89531966D
:1006E00000200895FBDF202DF9DF302DF7DF402DAE
:1006F000F5DF502D089582E001C084E099279D9395
:100700008A95E9F7089594E081918D939A95E1F7A0
:100710000895DD24863E6666A63F3D0AB73FE17A2E
:06072000943F14AE873F78
:00000001FF
